:103BF2000FC30FBF0FBB0FB60FB20FAC0FA70FA1B2
:103C02000F9B0F950F8E0F870F800F780F700F6825
:103C12000F5F0F550F4B0F410F360F2B0F1F0F1258
:103C22000F060EF80EEA0EDB0ECC0EBC0EAB0E9A91
:103C32000E880E750E620E4E0E390E240E0E0DF704
:103C42000DDF0DC70DAE0D940D790D5E0D410D24E6
:103C52000D070CE80CC90CA90C890C680C460C2346
:103C62000C000BDC0BB80B930B6E0B480B210AFA02
:103C72000AD30AAC0A840A5B0A330A0A09E109B7C1
:103C8200098E0965093B091108E808BE0895086C08
:103C92000842081907F107C807A007780750072943
:103CA200070206DB06B5068F066A0645062105FDF4
:103CB20005DA05B70595057405530532051204F3B7
:103CC20004D404B60498047B045F04430428040D5E
:103CD20003F303DA03C103A90391037A0363034DD8
:103CE20003370322030E02F902E602D302C002AE38
:103CF200029C028B027A026A025A024B023C022D99
:103D0200021F0211020301F601E901DD01D001C522
:103D120001B901AE01A30198018E0184017A0171FA
:103D22000168015F0156014D0145013D0135012E3A
:103D32000126011F01180111010B010400FE00F808
:103D420000F200EC00E600E100DC00D600D100CC7D
:103D520000C800C300BE00BA00B600010C01010495
:103D620002011E030A9604013205040406006407D8
:103D7200010108000009015A0E01010F00011200A1
:103D82006413010114013C1501FA1664FA17FFFFCE
:103D92001D00072000072400022701012F013C30EB
:103DA200010132010335FFFF3603073CFFFF3DFFF0
:103DB200FF180002191E461A00021B00022D32C80B
:063DC2002E0001FAFAFADE
:10004800900786E0FEA3E0FF7457BE0010D39F40E0
:100058000C903D5C12001EE493F59980129007867F
:10006800E0FEA3E0FF903D5C12001EE493F599903A
:10007800078612000E900786E0FEA3E0FF746C6FFF
:100088004E700375130022900072E0B402087401E8
:10009800900072F0D20C90013AE090002AF09001A2
:1000A8003BE090002BF090013CE090002CF0A20A7D
:1000B800B3401690013AE0700C90013BE070069056
:1000C800013CE060028002C20A90013AE0B4300FBD
:1000D80090013BE0B4470890013CE0643B6002803B
:1000E80004D20B8002C20BE557B40102800302025E
:1000F80011900057E0F565900062E0F567900063A5
:10010800E0F568900074E0F56990007AE0900029C5
:10011800F090007CE0F56490007DE0F5669000804A
:10012800E0F563900081E0F562900090E090004176
:10013800F0900091E0900042F0900092E09000432F
:10014800F0900093E0900044F0900094E090004517
:10015800F0900095E0900046F0900096E0900047FF
:10016800F0900097E0900048F0900099E0900033FC
:10017800F090009AE0900034F090009BE0900035F9
:10018800F090009CE0900036F0900079E0B4011700
:1001980090000A740FF0A374FFF090000CE4F0A331
:1001A800F07402900079F0900079E0B4035990005F
:1001B8000CE0FEA3E0FF90000AE0FCA3E0FD1200C3
:1001C800037410123F287408123F1AEF900026F0AB
:1001D800EF700674FF900026F07400900079F0909C
:1001E800000BE0900027F090000AE0900028F090C3
:1001F8000026E0900789F0900027E090078AF090A9
:100208000028E090078BF0803F900081E070067531
:100218005701756200A20AB3402E90013AE090009F
:100228002AF090013BE090002BF090013CE0900018
:100238002CF090002AE0700C90002BE070069000E3
:100248002CE060028002C20AE5657003756502E56C
:100258006770037567027E837FC2E5658E048F052C
:10026800FF123F0A8C388D39E56875F0FAA4FFAEA5
:10027800F0E5678E048F05FF123F0A8C3C8D3D9098
:10028800004FE0F55F90004DE0FE900069E0B50694
:100298001890004CE0FE900068E0B5060C90004B0A
:1002A800E0FE900059E06E606F900069E070069083
:1002B8000068E060067400900059F0900069E0B4AE
:1002C80002089000497401F08005900049E4F0901C
:1002D8000068E0B4020890004A7401F080059000BC
:1002E8004AE4F0900068E0600690004AE06002800E
:1002F80005755F038003755F04E558B55702D20C96
:10030800900068E090004CF0900069E090004DF09B
:10031800900059E090004BF0740090009EF074013A
:1003280090009FF074019000A0F074019000A1F07B
:1003380074009000A2F074009000A3F07400900084
:10034800A4F074009000A5F074019000A6F0740069
:100358009000A7F074019000A8F074009000A9F034
:1003680074009000AAF074009000ABF07400900044
:10037800ACF074019000ADF074019000AEF074011F
:100388009000AFF074009000B0F074009000B1F0ED
:1003980074009000B2F07400900362F0740190034E
:1003A80063F07401900364F07401900365F07400C5
:1003B800900366F07400900367F07400900368F08F
:1003C80074009003A2F074019003A3F074019003E9
:1003D800A4F074009003A5F074009003A6F07400D4
:1003E8009003A7F074009003A8F074009003E2F063
:1003F80074009003E3F074019003E4F07401900337
:10040800E5F074009003E6F074009003E7F07400E0
:100418009003E8F07401900422F07400900423F033
:100428007401900424F07400900425F07400900482
:1004380026F07400900427F07400900428F022E558
:10044800B554F7F5B5E5B554FDF5B5C2A2C2A1C2DC
:1004580092C207E5B554FBF5B5755004E55004F5AF
:100468005190004FE0F55F900025E4F0C209E5B532
:1004780054FEF5B522750A00750900AE09AF0A7475
:1004880057BE00039F500302053A903D5C12001EC0
:10049800E49390004E123F400FBF00010EE0FC9025
:1004A8003D5C12001EECFEE493FFEEC39F5026AEA7
:1004B80009AF0A0FBF00010E903D5C12001EAE0985
:1004C800AF0AE493FC903D5C12001EE49390004E4A
:1004D800123F40ECF0AE09AF0A903D5C12001EE4FA
:1004E8009390004E123F40E0FC903D5E12001EECDF
:1004F800FCE493FDECD39D4019903D5E12001EE490
:1005080093FC903D5C12001EE49390004E123F4015
:10051800ECF0AE09AF0A74022FFF50010E8E098F5E
:100528000A780A740126F6500418E436F6400302E5
:10053800048322750A00750900AE09AF0A7415BE56
:1005480000039F5003020608903DB312001EE49377
:1005580090004E123F400FBF00010EE0FC903DB3EB
:1005680012001EECFEE493FFEEC39F5026AE09AFC7
:100578000A0FBF00010E903DB312001EAE09AF0A6C
:10058800E493FC903DB312001EE49390004E123F9A
:1005980040ECF0AE09AF0A903DB312001EE4939010
:1005A800004E123F40E0FC903DB512001EECFCE40A
:1005B80093FDECD39D4019903DB512001EE493FCC9
:1005C800903DB312001EE49390004E123F40ECF0B1
:1005D800AE09AF0A740F6F4E7006750A15750900DB
:1005E800AE09AF0A74022FFF50010E8E098F0A78E8
:1005F8000A740126F6500418E436F6400302054151
:1006080022054C22054B22054DC2CF2290F800E46A
:10061800936406600280FE75840175A70075FF80EB
:10062800900788E4F075C91075A70F75A1C775A75D
:100638000075D90075CEFF75A70F75F1FE75F2FF2D
:1006480075F33775F47875A4BA75A5FF75A607759F
:10065800AE0075AFFF75D48175D5FF75D6FF75D718
:10066800FFC296C295C2A0C297E5B554BFF5B5E5DD
:10067800B554DFF5B5E5B554EFF5B5E5B5547FF5F7
:10068800B5E5B554F7F5B5E5B554FDF5B575A7006D
:1006980075A20175A14775F80975BC0175BE047589
:1006A800BD6C75BE0775BDA075BE0875BD0175BC6E
:1006B8000075BB1875BC2075BA0875E88075D1132C
:1006C80075A70F75E10575E20075C7407597007548
:1006D8009780740A123EFA7597C0E5975420700205
:1006E80080F8758F0275A700D2AF75980075A90CB0
:1006F80075A70F75AB4375ADFB75AC1E75A7007577
:100708008911758E00758C00758A00D2A9D28C75F6
:100718008D00758B00D2ABD28E75CD0075CC00756F
:10072800CA0075CB00D2ADC2CFD2CA7591047592FA
:10073800007593CD75EF0675D94075CF0190078682
:10074800E4F0A3F0751300751400C299D20A74C8B6
:10075800F51875170012251B75A70FE5FB90001AF1
:10076800F0E5FA90001BF0E5F990001CF075A70081
:1007780090F800E493F508122652122B8C90078902
:10078800E0900026F090078AE0900027F090078B11
:10079800E0900028F090078CE0900029F090078DF9
:1007A800E0F56590078EE0F56790078FE0F56890B3
:1007B8000790E0F569900791E0F564900792E0F5FD
:1007C80066900793E0F563900794E0F562900795CB
:1007D800E090002AF0900796E090002BF0900797A1
:1007E800E090002CF0900798E0900041F090079975
:1007F800E0900042F090079AE0900043F090079B49
:10080800E0900044F090079CE0900045F090079D30
:10081800E0900046F090079EE0900047F090079F18
:10082800E0900048F09007A0E0900033F09007A116
:10083800E0900034F09007A2E0900035F09007A314
:10084800E0900036F07400900082F090013AE07079
:100858000C90013BE0700690013CE060028004C20D
:100868000A8002D20A90F807E493900021F09000E1
:1008780021E0440A900021F0900021E054FE90000D
:1008880021F07406900012F07402900013F090F8B2
:1008980002E493900014F07403900015F074039030
:1008A8000016F07410900017F07405900018F0749A
:1008B80004900019F090F804E49390001DF074007F
:1008C80090001EF090F805E49390001FF090F80651
:1008D800E493900020F074FF900022F0744A900195
:1008E80025F07461900126F07474900127F0746308
:1008F800900128F0746F900129F0742090012AF07B
:10090800744A90012BF0745290012CF074349001C9
:100918002DF0743090012EF0743590012FF074454D
:10092800900130F07420900131F07434900132F06D
:100938007453900133F090007AE0D3940140067428
:100948000090007AF0755701755801740390004CB7
:10095800F012008F12047D12053B122547E5B554AD
:10096800FEF5B5900025E4F0900786E4F0A3F07555
:100978002300752200754700752900752800754801
:1009880000753100753000754900755300755400C5
:1009980075590075500475510175333C75320075F1
:1009A8006F00756E007570CD7555007556007542EF
:1009B80000754300754400754500755A007546007A
:1009C800754100754000900006E4F0A3F09000081F
:1009D800E4F0A3F0755D00755E0090000E74FDF004
:1009E800A374E8F0900023E4F07464900024F0C24B
:1009F80000D201C202D203754C00756C00C294C2C9
:100A080093C287C290C291C20C7E017F00900028D9
:100A1800E0123F28900027E02FFF50010E90000AB7
:100A2800EEF0A3EFF0900026E0700674FF90002629
:100A3800F090000AE0FEA3E0FFEFD394FFEE940FDE
:100A4800400790000AE4F0A3F07400900071F0747D
:100A580000900079F07400900082F0740090008D8E
:100A6800F074009000B4F0E5667003756604743A9B
:100A780090074EF074FD90074FF09003D4E0900477
:100A880014F0D2B0D2B7D2A7D2A6D2B1D2A3C2079D
:100A9800A2B6B39204A2B3B39205D29CD2EC75CF9E
:100AA80001A298B34005C298122EF0E5136006A281
:100AB80099B3B340028005C299123466E514640103
:100AC8006005E514B4040280D5E54CD39405400CC8
:100AD800E559C394C850020559754C00E570C39494
:100AE800F0501A786E12003FAE6EAF6FEFD394E8F5
:100AF800EE940340080570756F00756E00C28E7E17
:100B0800047F00E54B123F28E58D75F004A4FDAC89
:100B1800F0EF2DFDEE3CFCE58B75F04084FF7E0088
:100B2800ED2FFFEC3EFE8E248F25D28EA2B6300428
:100B380001B35003020C6CA2B6300401B350030297
:100B48000C6CA2B6405A0553E5B54401F5B59000C2
:100B580024E4F0E553D3956540447C837DC2123D7F
:100B6800C88E228F23E5472FFF50010E7401123FD4
:100B78001A8E228F23852347755301C28E758D00E7
:100B8800758B00754B00D28E7403BE00039F500610
:100B98009000257401F0E542B40603754200D204C2
:100BA800A2B6B35003020C6CC20490006BE060184C
:100BB8001235A7A200B34008E5B54408F5B580068C
:100BC800E5B554F7F5B58002C20090006EE06018F4
:100BD8001236FCA202B34008E5B54402F5B580061A
:100BE800E5B554FDF5B58006E5B554FDF5B5A207A4
:100BF800B34004D2878002C287900059E06004D2D3
:100C0800908002C29090004AE0B40104D29480021D
:100C1800C294900049E0B40104D2938002C293A226
:100C280009B34004D2918002C291900018E0FE906E
:100C38000014E0C39E4009900014E0D394084009D2
:100C480074FB900023F012044790001DE06015909B
:100C5800001DE0FE900017E06E600974FE9000230E
:100C6800F0120447C2CA7E017F00E54D123F28E515
:100C7800CD2FFF50010E8E268F27D2CAE564B4010E
:100C88004890000EE0FCA3E0FDEFC39DEE9C4039C8
:100C9800B208E52945286013A208B34008E5B54421
:100CA80004F5B58006E5B554FBF5B590000EE0FEF9
:100CB800A3E0FF900010E0FCA3E0FDEF2DFDEE3C6B
:100CC800FC90000EECF0A3EDF0A2B3300501B35098
:100CD80003020DB1A2B3300501B35003020DB1A256
:100CE800B35003020DAA0554E5B54401F5B59000CB
:100CF80024E4F0E554D395675003020DA87CEA7DFF
:100D080060AE26AF27123DC88E288F29E568123FAE
:100D18002874FF8E048F05FF123F0A8C288D29E561
:100D2800482DFD50010C74018C068D07123F1A8E58
:100D3800288F29852948A209B340157464123F28D1
:100D4800900067E08E048F05FF123F0A8C288D29DA
:100D580075540190000EE0FEA3E0FFAC26AD27120B
:100D6800000390000EEEF0A3EFF0E566FF123F0AD5
:100D7800740AFF123F0A90007BE08C068D07123F31
:100D88002874148E048F05FF123F0A900010ECF0AF
:100D9800A3EDF0C2CA75CD0075CC00754D00D2CA5E
:100DA800D205A2B3B34002C205900025E0B4010702
:100DB800E555C3940640030213C5E56C9024FAF880
:100DC800282873900059E0C394024003020F1FE5DE
:100DD80050D394015003020F1FE55075F040A4FF53
:100DE800AEF090031212001EE0C395445018E5506F
:100DF80075F040A4FFAEF090031112001EE0F52D2F
:100E0800752C00020F1FE55075F040A4FFAEF0905E
:100E1800031012001EE0C395444003020EBBE550C8
:100E280075F040A4FFAEF090031112001EE5507556
:100E3800F040A4FFAEF0E0FC90030F12001EECFEA1
:100E4800E0FFEEC39FFEE5508E0475F040A4FFAEB0
:100E5800F090031012001EE0F40425448C0088F082
:100E6800A4FFAEF0E5508F048E0575F040A4FFAEE8
:100E7800F090031212001EE55075F040A4FFAEF08A
:100E8800E0FA90031012001EEAFEE0FFEEC39FFE98
:100E9800CDCCCD8E07123F0AE55075F040A4FFAEC9
:100EA800F090030F12001EE02DFD50010C8C2C8DCC
:100EB8002D8064E55075F040A4FFAEF090030F124A
:100EC800001EE55075F040A4FFAEF0E0FC90030E64
:100ED80012001EECFEE0FFEEC39F8544F0A4FFAEB7
:100EE800F0E5508F048E0575F040A4FFAEF0900336
:100EF8001012001EE0FECDCCCD8E07123F0AE55041
:100F080075F040A4FFAEF090030E12001EE02DFD18
:100F180050010C8C2C8D2D756C010213C590005955
:100F2800E0C3940240030210D390004FE0D39550E1
:100F3800500302107BE55075F040A4FFAEF090031B
:100F48001812001EE0C395445018E55075F040A4EF
:100F5800FFAEF090031712001EE0F52B752A000271
:100F6800107BE55075F040A4FFAEF0900316120018
:100F78001EE0C395444003021017E55075F040A4E5
:100F8800FFAEF090031712001EE55075F040A4FF65
:100F9800AEF0E0FC90031512001EECFEE0FFEEC37D
:100FA8009FFEE5508E0475F040A4FFAEF090031646
:100FB80012001EE0F40425448C0088F0A4FFAEF073
:100FC800E5508F048E0575F040A4FFAEF09003182D
:100FD80012001EE55075F040A4FFAEF0E0FA900351
:100FE8001612001EEAFEE0FFEEC39FFECDCCCD8EAA
:100FF80007123F0AE55075F040A4FFAEF0900315C4
:1010080012001EE02DFD50010C8C2A8D2B8064E50A
:101018005075F040A4FFAEF090031512001EE55085
:1010280075F040A4FFAEF0E0FC90031412001EEC33
:10103800FEE0FFEEC39F8544F0A4FFAEF0E5508FBD
:10104800048E0575F040A4FFAEF090031612001E42
:10105800E0FECDCCCD8E07123F0AE55075F040A4D6
:10106800FFAEF090031412001EE02DFD50010C8C11
:101078002A8D2BE550B40123E55FD39401401CE58C
:101088005504D395504014E544C39405500D90037E
:101098005FE0A828B8000695294002800375500231
:1010A800E550B55F2290004FE0D395504019E550C8
:1010B80075F040A4FFAEF090031712001EE0A822BE
:1010C800B80006952340028002055F756C02021382
:1010D800C5900059E0B4022AE55075F040A4FFAE6F
:1010E800F090031712001EE0F52B752A00E55075E5
:1010F800F040A4FFAEF090030E12001EE0F52D752F
:101108002C00900059E0B4030F900051E0F52B75C6
:101118002A00752D00752C00756C030213C5E55067
:1011280075F040A4FFAEF090032012001EE0C395B6
:101138005940030211FB900049E07036E550D39402
:10114800014029AE22AF23AC2CAD2DEDD39FEC9EF0
:10115800401AE55075F040A4FFAEF090031E12004F
:101168001EE0A828B80005D3952950028002155022
:101178008034E550D394024029AE22AF23AC2CAD85
:101188002DEDD39FEC9E401AE55075F040A4FFAEBC
:10119800F090031E12001EE0A828B80005D3952978
:1011A800500280021550E550B55137E550C3955FA0
:1011B8005030E55504D395504028AE22AF23AC2AD1
:1011C800AD2BEFD39DEE9C4019E55075F040A4FF80
:1011D800AEF090031F12001EE0A828B8000695295B
:1011E800400280020550C292E55065516005C20771
:1011F800755900756C040213C5E55075F040A4FFDD
:10120800AEF090031A12001EE0B40117E55075F015
:1012180040A4FFAEF090032012001EE0240AC395FC
:101228005940030212D1752F64752E00A207B350DE
:101238000B900060E02405C3954440030212D1E5F9
:101248005075F040A4FFAEF090031D12001EE0C3DD
:1012580095444064E55075F040A4FFAEF090031C3F
:1012680012001EE55075F040A4FFAEF0E0FC9003BC
:101278001B12001EECFEE0FFEEC39F8544F0A4FFA6
:10128800AEF0E5508F048E0575F040A4FFAEF090E7
:10129800031D12001EE0FECDCCCD8E07123F0AE5DD
:1012A8005075F040A4FFAEF090031B12001EE02D15
:1012B800FD50010C8C2E8D2FAE22AF23AC2EAD2FFE
:1012C800EFD39DEE9C4002D207756C050213C5E56D
:1012D80050B40109900059E0C3940240030213A5D9
:1012E800900358E0D3954450030213A5900356E0A9
:1012F800C395445040900357E0FE900355E0F40432
:101308002EFE900356E0F40425448E0088F0A4FFD6
:10131800AEF0900358E0FC900356E0F4042C8E04E1
:101328008F05FF123F0A900355E02DFD50010C8CEC
:101338002A8D2B802C900355E0FE900354E0F40492
:101348002E8544F0A4FFAEF0900356E08E048F057E
:10135800FF123F0A900354E02DFD50010C8C2A8D9A
:101368002BE550C3955F5030E55504D39550402880
:10137800AE22AF23AC2AAD2BEFD39DEE9C4019E5EE
:101388005075F040A4FFAEF090031F12001EE0A8B5
:1013980028B800069529400280037550029000493C
:1013A800E0B40106E550640160028003755002E56F
:0D13B8005065516005C207755900756C0045
:1024FA00020DCB020F250210D90211260212010287
:02250A0012D7E6
:1013C500900050E02402A822B80007D395234002DC
:1013D500C207900025E0B40109900059E0C39403C9
:1013E500400302154D900049E0600302149CE5504E
:1013F500D394014034E55075F040A4FFAEF090035E
:101405001412001EE0A822B8001FD39523401AE548
:101415005075F040A4FFAEF090031F12001EE0A827
:1014250028B80005D39529500280021550E550D300
:101435009401402FE55075F040A4FFAEF0900312E3
:1014450012001EE0C39544501AE55075F040A4FF04
:10145500AEF090031E12001EE0A828B80005D39533
:1014650029500280021550E550D394014022E555DC
:1014750004C39550501AE55075F040A4FFAEF090A6
:10148500031E12001EE0A828B80005D395295002B6
:1014950080021550021542E550D394024034E550C0
:1014A50075F040A4FFAEF090031412001EE0A822D0
:1014B500B8001FD39523401AE55075F040A4FFAE40
:1014C500F090031F12001EE0A828B80005D3952947
:1014D500500280021550E550D39402402FE5507517
:1014E500F040A4FFAEF090031212001EE0C3954435
:1014F500501AE55075F040A4FFAEF090031E12009F
:101505001EE0A828B80005D3952950028002155081
:10151500E550D394024022E55504C39550501AE591
:101525005075F040A4FFAEF090031E12001EE0A817
:1015350028B80005D39529500280021550E550655D
:10154500516005C207755900900060E0D39544507D
:1015550009900054E0C395445002C207900059E039
:1015650070030217B2A2A5B34008A2A4B3400302B8
:10157500179BAE34AF357441D39F749C9E4005785C
:101585003412003FAE34AF35EFB48806EEB4130223
:101595008003021778A2A5500302163B900059E07C
:1015A500B4010B90004FE0D3955F4002055F9000BA
:1015B50059E0B40254E55075F040A4FFAEF0900335
:1015C5002012001EE0C39559503F90004FE0D3957F
:1015D500504021E55504D395504019E55075F0402C
:1015E500A4FFAEF090031412001EE0A822B8000676
:1015F500952340028002055090004FE0F55FE550CD
:1016050065516005C207755900900059E0B403267D
:1016150090004FE0D395504008E55504D3955050C0
:10162500028002055090004FE0F55FE5506551607E
:1016350005C207755900A2A45003021778900059F6
:10164500E0B4016E900049E07035E550D394014057
:1016550029E55075F040A4FFAEF090031E12001E60
:10166500E0A828B8000FD39529400A1550755900F0
:1016750085505F800385505F8003755F018033E58A
:1016850050D394024029E55075F040A4FFAEF09088
:10169500031E12001EE0A828B8000FD39529400AA2
:1016A500155075590085505F800385505F8003751F
:1016B5005F02900059E0D39401500302176CE55086
:1016C50075F040A4FFAEF090032012001EE0C39514
:1016D50059400302176C900049E07041E550D394DE
:1016E500014034E55075F040A4FFAEF090031112AF
:1016F500001EE0A822B8001FD39523401AE55075B7
:10170500F040A4FFAEF090031E12001EE0A828B81A
:101715000005D39529500280021550803FE550D32E
:1017250094024034E55075F040A4FFAEF0900311EB
:1017350012001EE0A822B8001FD39523401AE550D9
:1017450075F040A4FFAEF090031E12001EE0A8281D
:10175500B80005D39529500280021550E550655112
:101765006005C207755900E555B40704055D80039A
:10177500755D00E562B4010EAE34AF35EF644070BF
:1017850005EE649C6002800EA2A54003755701A278
:10179500A44003755702A2A5B3B35006A2A4B3B3E0
:1017A500400280067535007534000218A0A2A5B365
:1017B5004008A2A4B3400302188CAE34AF3574417F
:1017C500D39F749C9E4005783412003FAE34AF35EC
:1017D500EFB48806EEB41302800302188CA2A5406C
:1017E5006F900068E0605A90004AE0B401079000ED
:1017F5004AE4F0800690004A7401F090004AE070D7
:1018050005755F038003755F0490004AE0B4010429
:10181500D2948002C294E550B4041AE55075F040A4
:10182500A4FFAEF090031E12001EE0A828B8000524
:10183500D3952950028008755003C2077559008059
:1018450003755F04E555B40704055D8003755D0008
:10185500A2A44033900069E06021900049E0B40102
:1018650007900049E4F080069000497401F090006B
:1018750049E0B40104D2938002C293E555B407044C
:10188500055D8003755D00A2A5B3B35006A2A4B3A0
:10189500B340028006753500753400E5576558601C
:1018A50006900082E06003021A28C29C7514007538
:1018B5001300C2CAE55790250CF828287380121228
:1018C5002B8C800D122C658008122D3E8003122E64
:0118D50017FB
:0F250C000218C20218C40218C90218CE0218D34E
:1018D600900029E090007AF0E565900057F0E56702
:1018E600900062F0E568900063F0E569900074F09E
:1018F600E56490007CF0E56690007DF0E56390007D
:1019060080F0E562900081F090002AE090013AF0C4
:1019160090002BE090013BF090002CE090013CF011
:10192600900041E0900090F0900042E0900091F02D
:10193600900043E0900092F0900044E0900093F015
:10194600900045E0900094F0900046E0900095F0FD
:10195600900047E0900096F0900048E0900097F0E5
:10196600900033E0900099F0900034E090009AF0F7
:10197600900035E090009BF0900036E090009CF0DF
:101986007400900082F0744A900125F07461900111
:1019960026F07474900127F07463900128F0746F38
:1019A600900129F0742090012AF0744A90012BF0DE
:1019B600745290012CF0743490012DF07430900123
:1019C6002EF0743590012FF07445900130F074209C
:1019D600900131F07434900132F07453900133F079
:1019E6009003D4E0900414F0743A90074EF074FD1E
:1019F60090074FF012008F900004E4F0A3F09000DF
:101A0600067475F0A37430F09000087475F0A37432
:101A160030F0855758D2CA754B00D29C741B900083
:101A260023F0E555C394065005E550B55103021A57
:101A3600C8C207E55075F040A4FFAEF0900322122D
:101A4600001EE030E003D38001C39296E55075F0A6
:101A560040A4FFAEF090032312001EE030E003D353
:101A66008001C39295E555B40106E5506401600214
:101A76008004C2A08019E55075F040A4FFAEF09036
:101A8600032412001EE030E003D38001C392A0E5D8
:101A96005075F040A4FFAEF090032512001EE03012
:101AA600E003D38001C39297855051AE28AF2974C5
:101AB60005BE00039F5007E544D3940550028002FB
:101AC600D292E555D394055003021C15C207E55082
:101AD600D394015003021B6AE55075F040A4FFAE93
:101AE600F090031E12001EE0A828B80007D395291F
:101AF60040021550E55065516067E55075F040A409
:101B0600FFAEF090032212001EE030E003D3800106
:101B1600C39296E55075F040A4FFAEF090032312F1
:101B2600001EE030E003D38001C39295E55075F0C6
:101B360040A4FFAEF090032412001EE030E003D371
:101B46008001C392A0E55075F040A4FFAEF090036B
:101B56002512001EE030E003D38001C39297855022
:101B660051021C15E555B406349000ACE030E00394
:101B7600D38001C392969000ADE030E003D380019C
:101B8600C392959000AEE030E003D38001C392A0EB
:101B96009000AFE030E003D38001C39297E555B4DF
:101BA60007349000A5E030E003D38001C3929690FD
:101BB60000A6E030E003D38001C392959000A7E031
:101BC60030E003D38001C392A09000A8E030E00388
:101BD600D38001C39297E555B4083490009EE03057
:101BE600E003D38001C3929690009FE030E003D3D8
:101BF6008001C392959000A0E030E003D38001C33A
:101C060092A09000A1E030E003D38001C3929790A8
:101C16000072E06058E54475F00284FF7E00900192
:101C26004E12001EE0F55BE54675F00A84FF7E0065
:101C360090024E12001EE0F55CE55B255CD39464D1
:101C4600400BE55B255CC39464F55B8003755B0024
:101C5600E55B75F00284FF7E008F5BEFC394335023
:101C660007EF24CDF55B8003755BFF801CE54475AB
:101C7600F00284FF7E0090014E12001EE075F00215
:101C860084FF7E00EF24CDF55BE595C3955B4004AC
:101C9600C2A28002D2A2A207B34005E555B407034B
:101CA6007570CDE595C395704004C2A18002D2A19E
:101CB600E542C3940640030222B9A2EDB3500302E3
:101CC60022B9C2EDE5426003021E1B7E017F00E5DC
:101CD600BE123F28E5BD2FFF50010E900000EEF02A
:101CE600A3EFF0900029E0B401177E0F7FFF90006C
:101CF60000E0FCA3E0FD120003900000EEF0A3EF6D
:101D0600F0900079E0B4025B900000E0FEA3E0FFF3
:101D160090000AE0FCA3E0FDEDD39FEC9E400F90FF
:101D26000000E0F8A3E090000AC8F0A3C8F0900015
:101D360000E0FEA3E0FF90000CE0FCA3E0FDEFD383
:101D46009DEE9C400F900000E0F8A3E090000CC8C8
:101D5600F0A3C8F0900000E0FEA3E0FF7404123F79
:101D66001A8F43900079E07060900000E0FEA3E0D7
:101D7600FF90000AE0FCA3E0FDEFD39DEE9C400D32
:101D8600120003900000EEF0A3EFF0800790000031
:101D9600E4F0A3F0900000E0FEA3E0FF7410123F11
:101DA60028900026E08E048F05FF123F0A9000005F
:101DB600ECF0A3EDF07400D39D74019C40089000F4
:101DC60001E0F54380037543FFE54375F00AA4FF80
:101DD600AEF074198E048F05FF123F0A8D44ED256F
:101DE60031FFAE3050010E7401123F1A8F44854404
:101DF60031753000EFD394624003754462900072EF
:101E0600E064016006900066E060028005754201AC
:101E1600800375BB17E542B401028003021F0B7EE7
:101E2600017F00E5BE123F28E5BD2FFF50010E9051
:101E36000000EEF0A3EFF0900072E0B4017EE5330F
:101E460045326025AC32AD331DBDFF011C8F028EBD
:101E5600038C068D07903BF212002EE493FE74016C
:101E660093FFEFC39AEE9B400280057832123F52F1
:101E7600AE32AF3374B3BE0025D39F40219000002D
:101E8600E0FCA3E0FD0FBF00010E903BF212002E16
:101E9600E493FE740193FFEDC39FEC9E4002800520
:101EA600783212003FAE32AF33E569123F287464D0
:101EB6008E048F05FF123F0A8D468033900066E040
:101EC600602D900000E0FEA3E0FFEFD39400EE94B7
:101ED60008400F900066E0B40104C2098002D209EE
:101EE600800D900066E0B40104D2098002C2099018
:101EF6000072E064026006900066E0600575BB163D
:101F06008003754202E542B402028003021FF97E95
:101F1600017F00E5BE123F28E5BD2FFF50010E9060
:101F26000000EEF0A3EFF0900072E0B4027EE5331D
:101F360045326025AC32AD331DBDFF011C8F028ECC
:101F4600038C068D07903A8812002EE493FE7401E6
:101F560093FFEFC39AEE9B400280057832123F5200
:101F6600AE32AF3374B3BE0025D39F40219000003C
:101F7600E0FCA3E0FD0FBF00010E903A8812002E90
:101F8600E493FE740193FFEDC39FEC9E400280052F
:101F9600783212003FAE32AF33E569123F287464DF
:101FA6008E048F05FF123F0A8D468033900066E04F
:101FB600602D900000E0FEA3E0FFEFD39400EE94C6
:101FC60008400F900066E0B40104C2098002D209FD
:101FD600800D900066E0B40104D2098002C2099027
:101FE6000072E07003754600900066E07002C20958
:101FF60075BB1FE542B403457E017F00E5BE123F77
:1020060028E5BD2FFF50010E900000EEF0A3EFF083
:102016007409123F2874E68E048F05FF123F0A8C5E
:10202600408D41E5492DFD50010C74018C068D074C
:10203600123F1A8E408F4185414975BB19E542B45E
:10204600040280030221A17E017F00E5BE123F2823
:10205600E5BD2FFF50010E900000EEF0A3EFF074E7
:1020660004123F1A8F4AE563B40102800302212E4F
:10207600756A00756A00E56AD39407400302211B5E
:10208600E56A900041123F40E0D3954A501AE56A4E
:10209600900041123F40E0F404254AFEE56A9000B4
:1020A60037123F40EEF08017E56A900041123F403C
:1020B600E0C3954AFEE56A900037123F40EEF0E530
:1020C6006AC394044009900084E0C3956A503BE5D6
:1020D6006A6029E56A900037123F40FEE0FFEE9005
:1020E600003FE0D39F4013E56A900037123F40E07F
:1020F60090003FF0E56A900040F0800E900037E0D7
:1021060090003FF07400900040F0786A740126F663
:10211600400302207C900040E0F4042408F555E5D5
:1021260055D394054002C292E563D39401402FE54E
:102136004AD3946E4004D20D8002C20D755505E552
:1021460063B40205A20DB340028003755507E5632B
:10215600B40306A20DB3B340028003755507E556D6
:1021660065556008E55004F551855556E555B407A3
:1021760008E5B54480F5B58006E5B5547FF5B5E5C7
:102186005564066005E555B40808E5B54410F5B58F
:102196008006E5B554EFF5B575BB13E542B4050207
:1021A60080030222B57E017F00E5BE123F28E5BD11
:1021B6002FFF50010E900000EEF0A3EFF074041212
:1021C6003F1A8F45E562B4020280030222B2756AA5
:1021D60000756A00E56AD394034003022269E56A42
:1021E600900033123F40E0D39545501AE56A9000BF
:1021F60033123F40E0F4042545FEE56A90002D12B7
:102206003F40EEF08017E56A900033123F40E0C38E
:102216009545FEE56A90002D123F40EEF0E56A60B6
:1022260029E56A90002D123F40FEE0FFEE90003156
:10223600E0D39F4013E56A90002D123F40E09000E6
:1022460031F0E56A900032F0800E90002DE09000AB
:1022560031F07400900032F0786A740126F640037B
:102266000221DA900082E07043E52945286036E5D0
:1022760057C39403500A900032E004C3940340020B
:102286008007900032E004F557E557D39402400AE0
:10229600900032E004D3940250028007900032E0AE
:1022A60004F5578007900032E004F55775BB180512
:1022B60042D2ECE55DD3940450030223D375CF01DB
:1022C600C2A2AE34AF357488D39F74139E4005A264
:1022D600A5B34014AE34AF357488D39F74139E40B3
:1022E60005A2A4B340028048783412003FAE34AF52
:1022F60035EFB4883BEEB41337A2A5B3500990006E
:102306004FE0D395505002800405508011A2A5B32A
:10231600500890004FE0655060028002D207A2A4E8
:10232600B35007E550D39401500280041550C207FC
:10233600A2A5B3B35006A2A4B3B340028006753576
:1023460000753400E55065516067E55075F040A4AE
:10235600FFAEF090032212001EE030E003D38001AE
:10236600C39296E55075F040A4FFAEF09003231299
:10237600001EE030E003D38001C39295E55075F06E
:1023860040A4FFAEF090032412001EE030E003D319
:102396008001C392A0E55075F040A4FFAEF0900313
:1023A6002512001EE030E003D38001C392978550CA
:1023B60051A20740057570CD80037570FFE595C382
:1023C60095704004C2A18002D2A10222C3AE24AFFE
:1023D60025EFD39420EE944E50030224CE120447E8
:1023E600C28E758D00758B00754B00D28EC2077537
:1023F6006F00756E007570CD7550047523007522DB
:1024060000755300755900C287900059E06004D2E8
:10241600908002C29090004AE0B40104D2948002F7
:10242600C294900049E0B40104D2938002C293A200
:1024360009B34004D2918002C29190006BE060180B
:102446001235A7A200B34008E5B54408F5B58006E5
:10245600E5B554F7F5B58002C20090006EE060184D
:102466001236FCA202B34008E5B54402F5B5800673
:10247600E5B554FDF5B58006E5B554FDF5B5900016
:102486000E74FDF0A374E8F0E542B406037542004D
:10249600900025E4F0752500752400758D00758B78
:1024A60000754B00900024E0C3940350089000246C
:1024B600E004F080067403900024F0900024E0B459
:1024C6000306E5B554FEF5B5AE26AF27EFD3941057
:1024D600EE9427401CC2CA75CD0075CC0075270046
:1024E600752600D2CA754D007529007528007554E9
:0424F60000020AA630
:1038AE00000001000132016401960196020002122D
:1038BE0002240200020003000340038003C0040040
:1038CE000440048004C00500060006000600060041
:1038DE00060006000600060000FF01310163019597
:1038EE0001FF01FF0211022302FF02FF02FF033F4D
:1038FE00037F03BF03FF043F047F04BF04FF05FFE4
:10390E0006FF06FF06FF06FF06FF06FF06FF06FF81
:10391E000FAA0FA50F9F0F9A0F940F8D0F870F8071
:10392E000F780F710F680F600F570F4E0F450F3B3B
:10393E000F300F250F1A0F0E0F020EF50EE80EDBCD
:10394E000ECC0EBE0EAE0E9F0E8E0E7D0E6C0E5A51
:10395E000E470E340E200E0C0DF70DE20DCB0DB5ED
:10396E000D9D0D850D6D0D540D3A0D200D050CE9B7
:10397E000CCE0CB10C940C760C580C3A0C1B0BFBA9
:10398E000BDB0BBB0B9A0B790B570B350B130AF199
:10399E000ACE0AAB0A870A640A400A1C09F809D43F
:1039AE0009B0098C09670943091F08FB08D608B23C
:1039BE00088E086A0846082307FF07DC07B9079632
:1039CE0007730751072F070D06EC06CA06AA0689CC
:1039DE0006690649062A060A05EC05CD05B00592CC
:1039EE0005750558053C0520050504EA04CF04B508
:1039FE00049C04820469045104390422040B03F468
:103A0E0003DE03C803B2039D038903750361034DEF
:103A1E00033B03280316030402F202E102D102C0A3
:103A2E0002B002A00291028202730265025702499D
:103A3E00023C022F02220216020901FD01F201E6EA
:103A4E0001DB01D001C601BB01B101A7019D0194AB
:103A5E00018B0182017901700168016001580150EA
:103A6E000148014101390132012B0125011E0118C6
:103A7E000111010B010500FF00FA0FA60FA00F990F
:103A8E000F920F8B0F840F7C0F740F6B0F620F58FA
:103A9E000F4E0F430F380F2C0F1F0F120F050EF77F
:103AAE000EE80ED80EC80EB70EA50E930E800E6C35
:103ABE000E580E420E2C0E150DFD0DE40DCB0DB154
:103ACE000D950D790D5D0D3F0D200D010CE10CC016
:103ADE000C9E0C7C0C590C350C100BEA0BC40B9E77
:103AEE000B760B4F0B260AFD0AD40AAA0A800A553A
:103AFE000A2A09FF09D409A8097C0950092508F9E1
:103B0E0008CD08A10875084A081E07F307C8079DC7
:103B1E0007730749072006F706CE06A6067E065748
:103B2E000630060A05E405BF059B057705540532E8
:103B3E00051004EF04CE04AE048F04710453043553
:103B4E00041903FD03E203C703AD0394037B036370
:103B5E00034B0334031E030802F302DE02CA02B64D
:103B6E0002A30291027F026D025C024C023C022C07
:103B7E00021D020E020001F201E401D701CA01BECC
:103B8E0001B101A6019A018F0185017A01700166CA
:103B9E00015D0153014A0141013901310129012120
:103BAE0001190112010B010400FD00F700F000EAFB
:103BBE0000E400DE00D900D300CE00C900C400BF6F
:103BCE0000BA00B500B100AD00A800A400A0009C92
:103BDE00009900950091008E008A00870084008174
:043BEE00007E007BDA
:10251B00751A00751900AE19AF1AAC17AD18EDC3CB
:10252B009FEC9E401674FF123EFA75CF01781A7419
:10253B000126F6500418E436F650DB22900786E4A9
:10254B00F0A3F0751000750F00751300751400C221
:10255B000ED20F22C2AF75D900758F0375B7A57553
:10256B00B7F190F800E4F0758F0175B7A575B7F169
:10257B00E50890F800F075B7A575B7F190F801E490
:10258B00F075B7A575B7F190079DE090F802F0755F
:10259B00B7A575B7F19007A1E090F803F075B7A553
:1025AB0075B7F190079EE090F804F075B7A575B775
:1025BB00F190079FE090F805F075B7A575B7F1900E
:1025CB0007A0E090F806F075B7A575B7F19007A2D4
:1025DB00E090F807F0758F0075D940D2AF229007C5
:1025EB0088E0B4AB61C2AF75D90075B62275F52220
:1025FB00758F0375B7A575B7F1740090F600F0757C
:10260B008F01750A00750900AE09AF0A7413BE007D
:10261B00279F402475B7A575B7F190078912001E47
:10262B00E0FC90F60012001EECF0780A740126F61E
:10263B00500418E436F650D0758F0075F51175B649
:10264B002075D940D2AF22C2AF75D90075F522756E
:10265B000A00750900AE09AF0A7413BE00229F4031
:10266B001F90F60012001EE493FC90078912001EC7
:10267B00ECF0780A740126F6500418E436F650D5BF
:10268B0075F51175D940D2AF22900788E0B4AA0234
:10269B0080030227D1C2AF75D90075B62275F5221A
:1026AB00758F0375B7A575B7F1740090EE00F075D3
:1026BB00B7A575B7F1740090F000F075B7A575B7B5
:1026CB00F1740090F200F075B7A575B7F174009036
:1026DB00F400F0758F01750A00750900AE09AF0A99
:1026EB0074FFC39F74019E402475B7A575B7F19015
:1026FB00004E12001EE0FC90EE0012001EECF07873
:10270B000A740126F6500418E436F650CF750A0009
:10271B00750900AE09AF0A74FFC39F74019E402474
:10272B0075B7A575B7F190024E12001EE0FC90F044
:10273B000012001EECF0780A740126F6500418E41F
:10274B0036F650CF750A00750900AE09AF0A74FF53
:10275B00C39F74019E402475B7A575B7F190044EC5
:10276B0012001EE0FC90F20012001EECF0780A74CE
:10277B000126F6500418E436F650CF750A00750999
:10278B0000AE09AF0A74FFC39F74019E402475B756
:10279B00A575B7F190064E12001EE0FC90F40012E6
:1027AB00001EECF0780A740126F6500418E436F695
:1027BB0050CF758F0075F51175B62075D940D2AF16
:1027CB00743A90074EF022900788E0B4AA02800377
:1027DB0002290FC2AF75D90075B62275F522758F18
:1027EB000375B7A575B7F1740090E600F075B7A542
:1027FB0075B7F1740090E800F075B7A575B7F17473
:10280B000090EA00F075B7A575B7F1740090EC0075
:10281B00F0758F01750A00750900AE09AF0A74FFD8
:10282B00C39F74019E402475B7A575B7F190004EF8
:10283B0012001EE0FC90E60012001EECF0780A7409
:10284B000126F6500418E436F650CF750A007509C8
:10285B0000AE09AF0A74FFC39F74019E402475B785
:10286B00A575B7F190024E12001EE0FC90E8001225
:10287B00001EECF0780A740126F6500418E436F6C4
:10288B0050CF750A00750900AE09AF0A74FFC39FDC
:10289B0074019E402475B7A575B7F190044E1200D4
:1028AB001EE0FC90EA0012001EECF0780A74012680
:1028BB00F6500418E436F650CF750A00750900AED1
:1028CB0009AF0A74FFC39F74019E402475B7A575A9
:1028DB00B7F190064E12001EE0FC90EC0012001EA9
:1028EB00ECF0780A740126F6500418E436F650CF53
:1028FB00758F0075F51175B62075D940D2AF743A46
:10290B0090074EF022900788E0B4AA028003022AB7
:10291B004DC2AF75D90075B62275F522758F03754B
:10292B00B7A575B7F1740090DE00F075B7A575B754
:10293B00F1740090E000F075B7A575B7F1740090D5
:10294B00E200F075B7A575B7F1740090E400F0756F
:10295B008F01750A00750900AE09AF0A74FFC39F9A
:10296B0074019E402475B7A575B7F190004E120007
:10297B001EE0FC90DE0012001EECF0780A740126BB
:10298B00F6500418E436F650CF750A00750900AE00
:10299B0009AF0A74FFC39F74019E402475B7A575D8
:1029AB00B7F190024E12001EE0FC90E00012001EE8
:1029BB00ECF0780A740126F6500418E436F650CF82
:1029CB00750A00750900AE09AF0A74FFC39F740145
:1029DB009E402475B7A575B7F190044E12001EE00A
:1029EB00FC90E20012001EECF0780A740126F650FF
:1029FB000418E436F650CF750A00750900AE09AF1E
:102A0B000A74FFC39F74019E402475B7A575B7F177
:102A1B0090064E12001EE0FC90E40012001EECF03B
:102A2B00780A740126F6500418E436F650CF758FE9
:102A3B000075F51175B62075D940D2AF743A900771
:102A4B004EF022900788E0B4AA028003022B8BC2BF
:102A5B00AF75D90075B62275F522758F0375B7A5BD
:102A6B0075B7F1740090D600F075B7A575B7F17412
:102A7B000090D800F075B7A575B7F1740090DA0027
:102A8B00F075B7A575B7F1740090DC00F0758F0188
:102A9B00750A00750900AE09AF0A74FFC39F740174
:102AAB009E402475B7A575B7F190004E12001EE03D
:102ABB00FC90D60012001EECF0780A740126F6503A
:102ACB000418E436F650CF750A00750900AE09AF4D
:102ADB000A74FFC39F74019E402475B7A575B7F1A7
:102AEB0090024E12001EE0FC90D80012001EECF07B
:102AFB00780A740126F6500418E436F650CF750A9E
:102B0B0000750900AE09AF0A74FFC39F74019E40A4
:102B1B002475B7A575B7F190044E12001EE0FC901A
:102B2B00DA0012001EECF0780A740126F650041835
:102B3B00E436F650CF750A00750900AE09AF0A747A
:102B4B00FFC39F74019E402475B7A575B7F190061E
:102B5B004E12001EE0FC90DC0012001EECF0780A16
:102B6B00740126F6500418E436F650CF758F0075B5
:102B7B00F51175B62075D940D2AF743A90074EF067
:102B8B0022C2AF75D90075F522750A00750900AE22
:102B9B0009AF0A74FFC39F74019E401F90EE001291
:102BAB00001EE493FC90004E12001EECF0780A74A9
:102BBB000126F6500418E436F650D4750A00750950
:102BCB0000AE09AF0A74FFC39F74019E401F90F0C3
:102BDB000012001EE493FC90024E12001EECF078E3
:102BEB000A740126F6500418E436F650D4750A0020
:102BFB00750900AE09AF0A74FFC39F74019E401F95
:102C0B0090F20012001EE493FC90044E12001EEC96
:102C1B00F0780A740126F6500418E436F650D47591
:102C2B000A00750900AE09AF0A74FFC39F74019EB9
:102C3B00401F90F40012001EE493FC90064E12000D
:102C4B001EECF0780A740126F6500418E436F650A0
:102C5B00D475F51175D940D2AF22C2AF75D90075B5
:102C6B00F522750A00750900AE09AF0A74FFC39F00
:102C7B0074019E401F90E60012001EE493FC90002E
:102C8B004E12001EECF0780A740126F6500418E47C
:102C9B0036F650D4750A00750900AE09AF0A74FFF9
:102CAB00C39F74019E401F90E80012001EE493FC2A
:102CBB0090024E12001EECF0780A740126F65004B6
:102CCB0018E436F650D4750A00750900AE09AF0A40
:102CDB0074FFC39F74019E401F90EA0012001EE414
:102CEB0093FC90044E12001EECF0780A740126F649
:102CFB00500418E436F650D4750A00750900AE0975
:102D0B00AF0A74FFC39F74019E401F90EC0012002A
:102D1B001EE493FC90064E12001EECF0780A740130
:102D2B0026F6500418E436F650D475F51175D940D3
:102D3B00D2AF22C2AF75D90075F522750A0075099D
:102D4B0000AE09AF0A74FFC39F74019E401F90DE53
:102D5B000012001EE493FC90004E12001EECF07863
:102D6B000A740126F6500418E436F650D4750A009E
:102D7B00750900AE09AF0A74FFC39F74019E401F13
:102D8B0090E00012001EE493FC90024E12001EEC29
:102D9B00F0780A740126F6500418E436F650D47510
:102DAB000A00750900AE09AF0A74FFC39F74019E38
:102DBB00401F90E20012001EE493FC90044E1200A0
:102DCB001EECF0780A740126F6500418E436F6501F
:102DDB00D4750A00750900AE09AF0A74FFC39F745E
:102DEB00019E401F90E40012001EE493FC90064EDF
:102DFB0012001EECF0780A740126F6500418E43623
:102E0B00F650D475F51175D940D2AF22C2AF75D932
:102E1B000075F522750A00750900AE09AF0A74FF3B
:102E2B00C39F74019E401F90D60012001EE493FCBA
:102E3B0090004E12001EECF0780A740126F6500436
:102E4B0018E436F650D4750A00750900AE09AF0ABE
:102E5B0074FFC39F74019E401F90D80012001EE4A4
:102E6B0093FC90024E12001EECF0780A740126F6C9
:102E7B00500418E436F650D4750A00750900AE09F3
:102E8B00AF0A74FFC39F74019E401F90DA001200BB
:102E9B001EE493FC90044E12001EECF0780A7401B1
:102EAB0026F6500418E436F650D4750A007509005E
:102EBB00AE09AF0A74FFC39F74019E401F90DC00E4
:102ECB0012001EE493FC90064E12001EECF0780AE2
:102EDB00740126F6500418E436F650D475F51175C6
:102EEB00D940D2AF22E51464046006E59964FF6013
:102EFB00028031A20E4004D20E8027E514600874C4
:102F0B00E62514900023F0E513600874F025139068
:102F1B000023F0E514B4010280FE75140075130054
:102F2B00C20E8002C20EE514903851F82828737532
:102F3B001400E599B4FF03751301E599B4FE03750D
:102F4B001302E599B4FD03751303E599B4FC0375FE
:102F5B001304E599B4FA03751305E599B4FB0675EB
:102F6B001401120447E599B4F906751404120447C9
:102F7B00E599D394E54007E599C394F04002801698
:102F8B008599157514027E017F00E515C394E61231
:102F9B003F288E0D8F0E900786E4F0A3F0E599D3B2
:102FAB0094C44007E599C394E6400280288599159F
:102FBB0075140374E5C39515F50E750D00AE0DAFC5
:102FCB000E9038AE12002EE493F87401939007869E
:102FDB00C8F0A3C8F0D299023465900786E0FEA32F
:102FEB00E0FFEFC39400EE94054009EFD394FFEE9E
:102FFB0094064013900786E0FEA3E0FF90004E126C
:10300B00001EE599F0800385996B90078612000EE0
:10301B00900786E0FEA3E0FFEFB40106EEB40702D3
:10302B00800302327290074EE0B43C0280030232FE
:10303B007275FFA0A20AB35005A20BB34003023175
:10304B0065C29C90007AE090078CF0900057E0905E
:10305B00078DF0900062E090078EF0900063E09097
:10306B00078FF0900074E0900790F090007CE09058
:10307B000791F090007DE0900792F0900080E09037
:10308B000793F0900081E0900794F090013AE09064
:10309B000795F090013BE0900796F090013CE09093
:1030AB000797F0900090E0900798F0900091E090D7
:1030BB000799F0900092E090079AF0900093E090BF
:1030CB00079BF0900094E090079CF0900095E090A7
:1030DB00079DF0900096E090079EF0900097E0908F
:1030EB00079FF0900099E09007A0F090009AE09075
:1030FB0007A1F090009BE09007A2F090009CE0905D
:10310B0007A3F07400900082F012008F74AB90074D
:0D311B0088F01225E974AA900788F0E557A6
:06385100022F3A022FE5F0
:10312800903872F82828738012122694800D12277E
:0B313800D280081229108003122A4EDA
:0F38720002312F02313102313602313B02314037
:10314300900788E4F090013AE0700C90013BE07046
:103153000690013CE060028004C20A8002D20A02A7
:103163003267C29C900078E0900789F090005EE09F
:1031730090078AF090005FE090078BF090007AE070
:1031830090078CF0900057E090078DF0900062E07C
:1031930090078EF0900063E090078FF0900074E04A
:1031A300900790F090007CE0900791F090007DE014
:1031B300900792F0900080E0900793F0900081E0F8
:1031C300900794F090013AE0900795F090013BE06E
:1031D300900796F090013CE0900797F0900090E004
:1031E300900798F0900091E0900799F0900092E09A
:1031F30090079AF0900093E090079BF0900094E082
:1032030090079CF0900095E090079DF0900096E069
:1032130090079EF0900097E090079FF0900099E050
:103223009007A0F090009AE09007A1F090009BE037
:103233009007A2F090009CE09007A3F07400900028
:1032430082F074AB900788F01225E974AA9007887E
:10325300F01226941227D2122910122A4ED29C75EC
:1032630099FB80FED29C7514007513007599FB02BF
:103273003465900786E0FEA3E0FFEF4E7006859964
:1032830010750F00900786E0FEA3E0FF74016F4EF8
:10329300701BAC0FAD10AA0DAB0EED2BFBEC3AFA85
:1032A3008A068B0790004E12001EE599F090078660
:1032B30012000E900786E0FEA3E0FF74026F4E70CB
:1032C3000C12008F8515997514007513000234656F
:1032D300900786E0FEA3E0FF90004E12001EE599E2
:1032E300F090078612000E900786E0FEA3E0FFAC85
:1032F3000DAD0E8F028E038C068D079038E61200FB
:103303002EE493F9740193FEEAD39EEB9940098569
:103313001599751400751300023465900786E0FE55
:10332300A3E0FF90004E12001EE599F0900786126D
:10333300000E900786E0FEA3E0FFEFB40006EEB4B4
:103343000102800302346575FFA090001CE0D39452
:10335300C7400B90001CE0C394C8F516801A900078
:103363001CE0D39463400B90001CE0C39464F516F7
:10337300800690001CE0F516E51675F002A4FFAE7A
:10338300F08F6AEF90004E123F40EFFCE0FDEC90AF
:103393000051123F40EDFCE0FDEC2DB51602800319
:1033A3000234570FEF90004E123F40E56AFFE0FCF6
:1033B300EF900052123F40ECFFE0FCEFC39CB516C8
:1033C300028003023457E56A900050123F40E56AD9
:1033D300FFE0FCEF900053123F40ECFFE0FCEF2CCA
:1033E300B51671E56A900054123F40E0C3951690FC
:1033F300079DF0E56A900055123F40E0C395169093
:10340300079EF0E56A900058123F40E0C39516907E
:10341300079FF0E56A900059123F40E0C39516906C
:1034230007A0F0E56A90005A123F40E0C39516905A
:1034330007A1F0E56A90005B123F40E0C395169048
:1034430007A2F012255F7599F975186475170012B4
:10345300251B80FE7599FF75186475170012251BCF
:0234630080FEE9
:093857000232750232D302331E65
:1034650022E513903860F82828730235A690078660
:10347500E0FEA3E0FF90001212001EE0F599900710
:103485008612000E900786E0FEA3E0FF74116F4ED2
:1034950070037513000235A68561990235A690075C
:1034A50086E0FEA3E0FF90004E12001EE0F599EFC6
:1034B500B40107EEB4070375130090078612000EDA
:0734C5000235A6900787E025
:0F38600002346F02347202349D0234A30234C862
:1034CC00903881F828287385239902359B85299992
:1034DC0002359B85439902359B85469902359B8520
:1034EC00509902359B855F9902359B85559902351C
:1034FC009B85579902359B756D00900069E07006AD
:10350C00900068E060028016A2A44006E56D4404B9
:10351C00F56DA2A54006E56D4402F56D801A90008C
:10352C004AE0B40106E56D4410F56D900049E0B435
:10353C000106E56D4420F56DA207B34006E56D4428
:10354C0001F56DA209B34006E56D4408F56D856D76
:10355C0099803CA20FB340077599FAC20F8017A24D
:10356C000CB3400575990F800B900023E0F59990F2
:10357C000023E4F0C20C80178541998012854A998A
:0F358C00800D85459980087599FC8003751300A3
:103881000234D30234D90234DF0234E50234EB02CC
:1038910034F10234F70234FD02350302355F02359B
:0D38A1008402358902358E02359302359878
:0B359B0090078612000E80031200480B
:03386F000235A37C
:1035A6002290006BE0B4010385231190006BE0B418
:1035B600020385291190006BE0B403038543119043
:1035C600006BE0B4040385461190006BE0B405037C
:1035D60085501190006BE0B4060385551190006B81
:1035E600E0B4070385571190006CE0FE90006DE093
:1035F600C39E500302367D90006BE0D39404402CAA
:1036060090006CE0D39511500990006DE0C39511C0
:1036160050028002D20090006CE0D39511500990C0
:10362600006DE0C395115002C200804990006BE026
:10363600B4041890006DE0C395115002D2009000BA
:103646006CE0D395114002C200802A90006CE0C362
:103656009511500990006DE0D3951150028002D269
:103666000090006CE0D39511500990006DE0C39571
:10367600115002C200807E90006BE0D39404402C6F
:1036860090006CE0C39511400990006DE0D3951150
:1036960040028002C20090006CE0C3951140099080
:1036A600006DE0D395114002D200804990006BE096
:1036B600B4041890006CE0C395115002C20090004B
:1036C6006DE0D395114002D200802A90006CE0C3D1
:1036D6009511400990006DE0D395114002D20090FB
:1036E600006CE0D39511400990006DE0C395114040
:1036F600028002C2002290006EE0B401038523110D
:1037060090006EE0B4020385291190006EE0B403C8
:103716000385431190006EE0B404038546119000C2
:103726006EE0B4050385501190006EE0B406038583
:10373600551190006EE0B4070385571190006FE0B5
:10374600FE900070E0C39E50030237D290006EE0F8
:10375600D39404402C90006FE0D39511500990004B
:1037660070E0C3951150028002D20290006FE0D340
:1037760095115009900070E0C395115002C2028065
:103786004990006EE0B40418900070E0C3951150A3
:1037960002D20290006FE0D395114002C202802A45
:1037A60090006FE0C395115009900070E0D3951119
:1037B60050028002D20290006FE0D395115009901A
:1037C6000070E0C395115002C202807E90006EE048
:1037D600D39404402C90006FE0C3951140099000EB
:1037E60070E0D3951140028002C20290006FE0C3E0
:1037F60095114009900070E0D395114002D20280E5
:103806004990006EE0B4041890006FE0C395115023
:1038160002C202900070E0D395114002D202802AC3
:1038260090006FE0C395114009900070E0D39511A8
:103836004002D20290006FE0D395114009900070CB
:0B384600E0C3951140028002C2022284
:093F40002582F58250020583225E
:10002E00EF2F500205832582F582E5833E2EF58360
:01003E00229F
:08000300C3EF9DFFEE9CFE22FD
:08003F000806B60002180622B3
:0D000E00A3E004F07006123F36E004F0227B
:083F52000816B6FF0218162242
:0E3F1A00048007C3CE13CECF13CFD5E0F6221E
:103DC800BC000FBE0008ED8FF084FFADF022E4FECA
:103DD800FF22BE000DEF60FE54F0606F20E7030283
:103DE8003E7EEAC0E0EBC0E078017A0075F001EEB3
:103DF80020E710EF25E0FFEE33FE0AC5F023C5F0FB
:103E080030E7F0EA5407F9096A7A007B0060010894
:103E1800C3EC9E40167004ED9F4010ED9FFDEC9E94
:103E2800FCE5F0CA4ACA03F5F08005E5F003F5F0B1
:103E3800C3EE13FEEF13FFD9D77908CACBCAD8D07F
:103E4800EAFEEBFFD0E0FBD0E0FA22EC8FF084FC36
:103E5800ED54F045F0C48FF084FEEDC454F045F005
:103E6800C48FF084FDEEC4FE54F02DFFEE540F3CD9
:103E7800FEADF07C0022790078008FF0EC7E0820FF
:103E8800E70DC3CD33CD33C933C9C833C8DEF08499
:103E980049F9E5F08FF0BE00E6FD7C00E9FFE8FE99
:013EA80022F7
:0E3F2800F88FF0A4FFE5F0CE88F0A42EFE2264
:103EFA00600D782B023F04007830D8FED5E0F82216
:103F0A00EEC0E07E00123DC8EFFDEEFCD0E0FE22DE
:03000B00023EA909
:03001B00023EC4DE
:03002B00023EDFB3
:03000000023F4973
:093F490075817175D000020614A7
:0B001E00E5822FF582E5833EF583228A
:0A3F36000582D58202158315822250
:103EA900C0E0C0F0C083C082C0D075D0001206093E
:103EB900D0D0D082D083D0F0D0E032C0E0C0F0C002
:103EC90083C082C0D075D00012060CD0D0D082D069
:103ED90083D0F0D0E032C0E0C0F0C083C082C0D04F
:103EE90075D00012060FD0D0D082D083D0F0D0E0A8
:013EF9003296
:00000001FF
